:10000000020C0700000C2700E802040AE902040AB7
:10001000520C2C008709530C2C008709540C2C001F
:100020008709F00C4C01500F4307110A0C020F0E08
:10003000E201290A2D0A310A320A330A3A0A410A30
:10004000410A420A460A4A0A4E0A4E0A4E0A4E0A15
:100050004F0A97090C020500110A97090C020600C5
:10006000110A000A000A05022C00870997090C02F0
:100070002500110A06022C00870997090C022600A8
:10008000110A000A05022C008709000A06022C004A
:100090008709110AAA0C2C008709110A000A6E00B0
:1000A0005809FF0E4306110A2C008709AE02500AB8
:1000B0000E02E201500849084308200831083608BA
:1000C000630838083408200845084D0855082008FA
:1000D00062086508740861082008760865087208D7
:1000E000730869086F086E082C08200862086C08FD
:1000F00061082C08200862086C0861082C08200898
:1001000062086C0861080A080A080D08000847051B
:10011000080C2B00A6092C03030647040307470518
:10012000A609EB028B0A47042C03A609000827073F
:10013000970A080C2B00AC09A60927060304270719
:1001400003052C03EB029C0AAC0900080F0C2A00E3
:100150000000EA02A80A0008080C2A000000EA02CF
:10016000AE0A0008FF0FFF0FFF0FFF0FFF0FFF0F7B
:100FF000FF0FFF0FFF0FFF0FFF0FFF0FFF0F000A85
:00000001FF
